:0400000500000000F7
:020000040000FA
:1000000018F09FE518F09FE518F09FE518F09FE5C0
:1000100018F09FE50000A0E120F11FE518F09FE532
:10002000540000004000000078150000440000006B
:1000300048000000000000004C00000050000000DC
:10004000FEFFFFEAFEFFFFEAFEFFFFEAFEFFFFEA18
:10005000FEFFFFEAF4009FE5AA10A0E35520A0E30D
:100060002030A0E3A03180E5A03190E5403013E2DC
:10007000FCFFFF0A0130A0E30C3180E50B30A0E368
:10008000843080E58C1080E58C2080E50130A0E391
:10009000803080E58C1080E58C2080E5883090E50C
:1000A000013313E2FCFFFF0A883090E5A0409FE592
:1000B000043003E00B40A0E3043033E0F9FFFF1A03
:1000C0000530A0E3043180E50530A0E3083180E588
:1000D0000A3DA0E3A83180E50238A0E3AC3180E519
:1000E0000330A0E3803080E58C1080E58C2080E533
:1000F00058009FE50410A0E3041080E50210A0E37F
:10010000001080E54C009FE5DBF021E300D0A0E18A
:10011000000040E2D7F021E300D0A0E1000040E27F
:10012000D1F021E300D0A0E1000040E2D2F021E3D1
:1001300000D0A0E1010C40E2D3F021E300D0A0E127
:10014000010C40E210F021E30C009FE510FF2FE1CD
:1001500000C01FE0FF7FFF00580800406001000062
:1001600000D09FE5D60400EB580600400047000091
:1001700010B40200002A01DB012A03DD0020C04385
:1001800010BC7047002A12D1E6480068F02398435B
:10019000E44B18601800006810231843E14B186006
:1001A0001800006840231843DE4B18601BE0DD4850
:1001B00000680F231B059843DA4B1860180000688D
:1001C00001231B051843D74B186018000068012352
:1001D0009B051843D34B1860D348406801231B0686
:1001E0001843D14B58600120A4235343CF4C1B1913
:1001F0005860A42050432300185808600120BFE72E
:100200000100012901DB022902DD0020C043704703
:10021000481EA4235843C54BC218481E06D1C148E6
:100220000068F0239843BF4B18600DE0BD4800689C
:100230000F231B059843BB4B1860BB484068012344
:100240001B069843B84B58600020136C1860B84BDD
:10025000106D5861002050600120D8E7FFB583B0D1
:1002600004001500012C01DB022C05DD0020C04339
:1002700007B0F0BC08BC1847601EA4235843AB4924
:100280004718052D06D0062D06D0072D06D0082DBF
:1002900007D105E0002606E0012604E0022602E080
:1002A000C0460326C046C0460C98002808D0012846
:1002B00002D0022805D100E0C0460420019003E0EE
:1002C000C04600200190C046C046069B01F0C6F81B
:1002D000051004070A0D1100082002900CE01820F8
:1002E000029009E02820029006E03820029003E006
:1002F000C04600200290C046C0460498B860FD6029
:100300000C9838610698786100219C20C151A0208A
:10031000C1518848049901F0AFF80009009000200D
:10032000796B0860802030430299084301990843A3
:10033000B96A08600098396A08600098000A796A0A
:10034000086030000299084301990843B96A0860BF
:100350008720B96B08600320396C0860012109040B
:10036000786D884340187865796CF86C08600F20C8
:10037000B96C08606E49386D0861012078E7F8B4FF
:100380000400012C01DB022C03DD0020C043F8BC7B
:100390007047601EA4235843644BC6181568106844
:1003A000A84201DD280000E010680500009514E077
:1003B000C046A02083599C2080598342F9D0A020B8
:1003C0008059A0239B595B1CA027BB5183069B0E21
:1003D00030005C30C05C0870491C28006D1E00288D
:1003E000E6D10098D3E7F7B40400012C01DB022C1E
:1003F00003DD0020C043FEBC7047601EA4235843A9
:100400004A4BC21802980668370014E0506DC003CA
:10041000C00F10D010250AE001200004536D834363
:1004200053650878D3691860491C761E6D1E002E2E
:1004300001D0002DF0D1002EE8D13800DBE710B458
:100440000400012C01DB022C03DD0020C04310BCA2
:100450007047601EA4235843344BC2189C20835815
:10046000A0208058181A8006800E08600120EEE750
:1004700010B40400012C01DB022C03DD0020C0437A
:1004800010BC7047601EA4235843284BC218542048
:10049000805A08800023542083520120F0E708B5D9
:1004A00025490120FFF764FE002200920822E12185
:1004B0004902214800680023FFF7D0FE01B008BCC4
:1004C000184701B582B0012001900D2000900298DC
:1004D0000A2805D101AA694617480068FFF783FF7B
:1004E00001AA02A914480068FFF77DFF029803B033
:1004F00008BC18470EB501200190C04602A90E485D
:100500000068FFF79CFF02980028F7D001AA69460F
:1005100009480068FFF733FF6B46187803B008BC42
:100520001847000000C002E0C0C01FE0000000400B
:1005300000F0FFFF00366E01480100400F502DE92A
:100540005C019FE53C2090E5001092E50F2001E260
:10055000020052E31400000A040052E30200000A01
:100560000C0052E31500001A010000EA0000A0E1AF
:100570000000A0E1070000EA182090E5002092E5C5
:100580009C3090E501C083E23F3003E29CC080E5EF
:100590005CC080E20320CCE72C2090E5002092E5AF
:1005A000010012E3F3FFFF1A060000EA0000A0E1D9
:1005B000542090E5012882E3542080E5010000EA00
:1005C0000000A0E10000A0E10000A0E12C2090E5E7
:1005D000002092E5CC309FE5032002E0B425C0E185
:1005E0000020A0E3002102E50F50BDE804F05EE228
:1005F0000F502DE9B0009FE53C2090E5001092E5FA
:100600000F2001E2020052E31400000A040052E34A
:100610000200000A0C0052E31500001A010000EA73
:100620000000A0E10000A0E1070000EA182090E52A
:10063000002092E59C3090E501C083E23F3003E268
:100640009CC080E55CC080E20320CCE72C2090E5D4
:10065000002092E5010012E3F3FFFF1A060000EA12
:100660000000A0E1542090E5012882E3542080E5B9
:10067000010000EA0000A0E10000A0E10000A0E10C
:100680002C2090E5002092E518309FE5032002E041
:10069000B425C0E10020A0E3002102E50F50BDE831
:1006A00004F05EE2000000401EE00000A4000040F4
:1006B00011C08FE21CFF2FE101000A07D00E80223B
:1006C000114200D0401C70471021EA4A916011008D
:1006D0000861C046E749096810221142FAD0704704
:1006E0001022E44B9A601A001061C046E14A126879
:1006F00010231A42FAD01022DE4B9A601A001161C0
:10070000C046DC4A126810231A42FAD07047010032
:100710003020D84A906010000161C046D54800687A
:1007200020221042FAD0D3484069704710B5040027
:10073000802020430004FF22013210430100CE48F4
:10074000FFF7CEFF802020430004FF220132104338
:100750000100C948FFF7C4FF10BC08BC18470020BF
:10076000C449403188604020C86001208860402032
:10077000C860C046BF480068FF2101310842F9D077
:100780000020C043BB498863486388600C204860F0
:1007900070477047704700B5B84840680F21890618
:1007A0008843B64948600800406805218906084327
:1007B000B24948600800C068B1490840AF49C86004
:1007C0000800C068AF490843AC49C8600800006928
:1007D000032189048843A9490861AB4800680121C5
:1007E00049020843A849086001204002C861A7489F
:1007F000406849060843A54948601220A449486357
:10080000C046A348806B122108401228F9D1A148A4
:10081000A14988610120A14988618005A04908613A
:10082000FFF79DFF0020FFF781FF08BC184710B5B8
:100830000400002C01D0012000E000200104FF2270
:10084000013211439748FFF74BFF10BC08BC184713
:1008500000B5954800880221084203D09349914889
:10086000FFF73EFF08BC1847704710B50400002C86
:1008700001D0012000E000200104FF2201321143D9
:100880008B48FFF72DFF03207A4940314860C0466E
:1008900078480068FF2101310842F9D0FF2001307B
:1008A0007449886010BC08BC184710B50400A078D3
:1008B000FFF702FF03006F48403041680120984075
:1008C00001436C48403041608360607921790002C7
:1008D000084368494031C860C04666480068FF2147
:1008E00001310842F9D0FF2001306249886010BC14
:1008F00008BC1847704730B504002000FFF7DCFE45
:1009000000046C49084305008913FFF7E9FE30BC79
:1009100008BC184730B504002000FFF7CDFE0004E6
:100920006449084305006449FFF7DAFE30BC08BC9F
:10093000184730B504002000FFF7BEFE00045D49F3
:10094000084305008913FFF7CBFE30BC08BC1847ED
:1009500030B504002000FFF7AFFE000455490843FE
:1009600005005249FFF7BCFE30BC08BC184730B543
:1009700004002000FFF7A0FE00044E4908430500D4
:100980008913FFF7ADFE30BC08BC1847F8B504006A
:100990000D002007800E401C36498862C04635484D
:1009A000066A0120C0020642F9D0B605B60D00273E
:1009B00006E030498869290000F07BFD2D1D7F1C71
:1009C000F01C8008B842F4D800202A4988623B48CD
:1009D0002041C007C00F0CD12000FFF76DFE0004BE
:1009E0000521090208430300FFF76EFE3448FFF7B4
:1009F0006BFE3000F8BC08BC1847F8B504000D00C9
:100A000016002007800E801C1A4988620800466282
:100A1000002706E0280000F043FD1649C8612D1D9F
:100A20007F1CF01C8008B842F4D80020114988626D
:100A30002000FFF741FE00040521090208430300DE
:100A4000FFF742FE1F48FFF73FFE3000F8BC08BC2E
:100A5000184700B51C48FFF737FE1C48FFF757FE44
:100A600003001A48FFF753FE00020343180008BCB6
:100A70001847000000C2E0FF0005D00000C002E0FF
:100A8000CFFFFFCF1000002040C0FF3FC0C01FE0DD
:100A9000C0CFE0FFD00A000040F1FFFF40F2FFFFAF
:100AA00000F0FFFF0005FE004C01004000010100C6
:100AB0000005D80000054000000120004812000099
:100AC0000005F2000005FA000005F5000002F5003F
:100AD000FF502DE978019FE5004290E5084280E54E
:100AE000080014E31400000A68019FE5EFFEFFEB25
:100AF00064019FE5BC0200EB0050A0E1100015E38B
:100B00000200000ABB0200EB660100EB4C0000EAA9
:100B1000020015E30000000A490000EA080015E39E
:100B20000500000A040015E30100000AB40200EB0E
:100B3000000000EAB50200EB410000EA040014E303
:100B40003E00000A390000EA0060A0E3350000EA38
:100B5000FC009FE5300290E50110A0E3110610E1D2
:100B60002E00000AA670A0E10100A0E31006A0E19B
:100B7000DC109FE5380281E50000A0E1D0009FE590
:100B8000000290E5200010E3FBFFFF0AC0009FE594
:100B9000145290E5010016E31700001A000056E316
:100BA0000B00001A040015E30900000AAC009FE5E1
:100BB000000090E5000050E30500000A9C009FE55E
:100BC000001090E50100A0E30FE0A0E111FF2FE18C
:100BD000130000EA84009FE5070190E7000050E35E
:100BE0000E00000A74009FE5071190E70200A0E3E1
:100BF0000FE0A0E111FF2FE1080000EA5C009FE593
:100C0000070190E7000050E30400000A4C009FE554
:100C1000071190E70300A0E30FE0A0E111FF2FE12F
:100C20000000A0E1016086E2200056E3C7FFFF3A22
:100C30001C009FE5300290E5000050E3C1FFFF1A61
:100C40000000A0E10000A0E3000100E5FF50BDE8C6
:100C500004F05EE200C0E0FF0005FE000002FE00BE
:100C6000601C00000020FF490880FF490870FF4910
:100C70000870FF48FF4908600020FF49086070477E
:100C800010B5FE490020FFF781FE10BC08BC1847D4
:100C900010B5FB488088402801DD402401E0F84879
:100CA0008488F74822000168802008DF0400F448A7
:100CB00000680019F249086008008088001B8880DD
:100CC00010BC08BC184710B5ED4801680020FFF7BC
:100CD0005DFE0400EA4800680019E9490860080060
:100CE0008088001B888010BC08BC184710B5002203
:100CF0001100802008DF10BC08BC184710B5E1497E
:100D00000020FFF743FE10BC08BC184710B50400D4
:100D1000230000F0A3FB08F805F7F6F8F8F5F4F85F
:100D2000FFF7AEFFD54909780906C80FFFF7E2FDC6
:100D3000D248C088D2498880D04800784006800FC9
:100D400004D001287CD002287BD111E1CB48437824
:100D500000F084FB0C070D8E168E1F30363D4B5D68
:100D60007D8E00F0B9FC002800D103E181E0002075
:100D700000F020FD002800D1FCE0FFF7B7FF78E08D
:100D8000012000F017FD002800D1F3E0FFF7AEFFCF
:100D90006FE0BA480078C006C00E08D1B748807826
:100DA00080210843B0490870FFF7A0FF00E0E1E0B0
:100DB000C0465EE000F032FC002800D1DAE058E0E6
:100DC0000020FFF7C5FD0020AD49888051E0AB4809
:100DD0000078C006C00E05D1A448A9490860FFF7F5
:100DE00057FF00E0C6E0C04643E0A4480078C006D4
:100DF000C00E09D100F052FD002800D1BAE0FFF783
:100E000075FF00F05BF900E0B4E0C04631E09B48BC
:100E10000078C006C00E012816D19448007800283A
:100E200010D0964800799849097888420ADA9348A0
:100E300000799649401892490860FFF729FF02E0BF
:100E400019E096E096E000E094E0C04611E08B489F
:100E50000078C006C00E012807D100F0EFFD002881
:100E600000D187E0FFF742FF00E083E0C04600E0EA
:100E700080E0C04685E081480078C006C00E0128A9
:100E800074D17E480079002803D07C48007901287D
:100E90006BD17A484078042837D008DC00280FD07E
:100EA000012811D002281AD003285DD11BE0202888
:100EB00035D0212837D0222840D0232854D147E0EC
:100EC00070486F49086052E000F0ABF9002805D087
:100ED0006C486B490860FFF7DBFE48E044E0694876
:100EE0006749086043E06549488800F09FF9002899
:100EF0000AD0644862490860FFF7CAFE37E0C7E0DD
:100F0000CAE095E03FE0CBE02EE05C49488800F085
:100F100090F9002802D0FFF7E9FE28E024E05948C4
:100F20005749086023E000F0BEF9002805D0554875
:100F300053490860FFF7ACFE19E015E04F494888B7
:100F400000F0D8F9002802D0FFF7D0FE0FE00BE048
:100F50004A49488800F0D1F9002804D0FFF7C6FEBE
:100F600005E003E001E0C046C04603E002E008E01F
:100F700000E0C0468020FFF7EBFC0020404988805D
:100F8000C046C0468CE03D4800780006C00F4CD1FA
:100F90003B48808800284AD0FFF795FE3848808873
:100FA000002844D1354800784006800F02D001283F
:100FB00036D100E0DEE731480078C006C00E0128D7
:100FC00002D0022829D127E02C480079002803D03C
:100FD0002A48007901281ED128484078002804D0EA
:100FE000022808D0202814D10DE000F018F90028BC
:100FF00000D1BFE70DE02149488800F014F900282E
:1010000000D1B7E705E000F017F9002800D1B1E7FB
:10101000C046C04602E0ADE7ACE7ABE7C04600E043
:10102000A8E7C046FFF762FE01E0FFF767FE37E082
:10103000124800780006C00F012802D1FFF728FEF1
:101040000EE0094800788021084209D0064800785F
:101050004006400E0449087008000078FFF766FB60
:101060001EE000004C0100404E0100404F010040D6
:10107000010001005001004054010040680100409F
:1010800060010040880100405801004059010040C3
:101090008020FFF76CFC03E00020FFF768FCC046EF
:1010A000C04610BC08BC184701C08FE21CFF2FE1EE
:1010B00010B5FFF7D7FD10BC08BC1847704770B5D6
:1010C0000500032D0BD100F02FF80400154801880E
:1010D000A14203D01348048000F03BF9C046C0464B
:1010E00070BC08BC184710B50400022C02D0032CB9
:1010F00006D102E000F01EF902E000F001F9C0465E
:10110000C04610BC08BC184770477047704770470E
:101110007047704770477047704770477047704717
:10112000704700007001004008B500209749088012
:10113000694697480068FFF79BF96B4618880121BC
:10114000C903084205D091480088012108438F490E
:1011500008806B46188801214903084205D08B4856
:10116000008802210843894908806B4618881021AD
:10117000084205D085480088042108438349088037
:101180006B46188801218903084205D07F480088F2
:10119000082108437D4908806B46188808210842C9
:1011A00005D07A48008810210843784908806B46AA
:1011B00018880421084205D074480088202108437B
:1011C000724908806B4618880221084205D06F4892
:1011D0000088402108436D4908806C48008801B0B0
:1011E00008BC184738B56A490020FEF7C1FF6948B6
:1011F00000F056F904006748027900924379827939
:10120000210063480068FFF729F80120624908803F
:10121000FFF78AFF5D49088038BC08BC18470120E9
:101220007047012070470100012070470100012034
:10123000704701000120704738B558490978574A6E
:10124000527812021143554A927812041143534ABC
:10125000D2781206114308004E4900F02AF94F488F
:1012600000794C4908714D48407948714B48807964
:10127000887147480068FEF7C3FF45490020FEF724
:1012800077FF444800F00CF90400424802790092CC
:101290004379827921003E480068FEF7DFFF012094
:1012A00038BC08BC184710B53A4800F0F9F83B497B
:1012B0000870384800F0F4F80004000E3749487010
:1012C000344800F0EDF80002000E344988703148CF
:1012D00000F0E6F8000E3149C8702E480079087118
:1012E0002C48407948712B4880798871012010BCC6
:1012F00008BC184701000120704701000120704719
:1013000038B5694622480068FFF799F86A462449CB
:101310001F480068FFF733F80400002C04DD2200AA
:101320001F49822008DF02E001201B49088038BCE9
:1013300008BC184708B51A490220FFF727FB0090A0
:101340006A46174912480068FFF74DF801B008BC1B
:10135000184710B5A12013490870202048700020BC
:101360008870C87008714871022088710020C871A7
:1013700006480088087205480088001248720A2250
:10138000812008DF10BC08BC184700007C01004029
:1013900080010040740100407E010040880100404F
:1013A000C80100400802004010B5FFF71BFF10BC49
:1013B00008BC184738B5694621480068FFF73FF870
:1013C0000098002811DD1F48008800280DD06A46CB
:1013D0001D491B480068FEF7D2FF04000020194990
:1013E000088022001849822008DF38BC08BC184752
:1013F00010B5FFF799FE040014480088A04203D0FE
:1014000012480480FFF7A5FF10BC08BC184710B5B0
:1014100000200F498862FF200E490860FFF7C4FFD3
:10142000FFF7B9F90120FFF702FAC0460A48007831
:101430000028FBD003E0FFF7BDFFFFF7D9FFFAE775
:10144000800100407E010040120200408401004003
:1014500000C002E040C0FF3F4F0100407847C04657
:1014600001C05EE50C0053E10330DE370C30DE27AF
:1014700083C08EE01CFF2FE10B00010030B4002080
:101480001F2201240D00D5409D4205D31D0095402B
:10149000491B250095404019521EF3D530BC7047BA
:1014A000021D0321521E137800021843491EF9D56C
:1014B0007047030003220870491C000A521EFAD527
:1014C0001800704701C08FE21CFF2FE1064C074D4A
:1014D00004E020000FC800F010F81034AC42F8D33C
:1014E0000348FEF743FE0000A01C0000C01C0000E3
:1014F0000F140000004708471047184720472847A7
:101500003047384710402DE902E081E001C0D0E4C7
:1015100007301CE20130D0044C22B0E10120D0049D
:10152000013053E20140D0140140C114FBFFFF1A07
:1015300008301CE20300001A012052E20130C154BD
:10154000FCFFFF5A060000EA0130D0E4022082E2EC
:10155000033041E0012052E201C0D35401C0C15424
:10156000FBFFFF5A0E0051E1E7FFFF3A1040BDE8D4
:101570000000A0E31EFF2FE100502DE900C04FE165
:1015800000112DE920001CE3B2C05E11FFCCCC138A
:1015900004C01E05FFC4CC0324809FE508005CE165
:1015A0000600002A1C808FE20CC198E70FE0A0E142
:1015B0001CFF2FE10011BDE80CF06FE10090FDE889
:1015C000FEFFFFEA09000000C0150000C015000082
:1015D000C0150000C0150000C0150000C0150000B7
:1015E000C0150000C0150000FB09000000C09FE509
:1015F0001CFF2FE10F07000000C09FE51CFF2FE13B
:101600005F07000000C09FE51CFF2FE19507000069
:1016100000C09FE51CFF2FE19307000070B529482B
:101620000078C006C00E02D001283DD139E025481F
:10163000C078012804D0022807D003282DD122E049
:10164000214822490860122529E0214C002608E0A3
:101650002078002804D0E078A1780002084304191B
:10166000761C18488078B042F2D12078002803D147
:10167000002070BC08BC184714480460E078A178CA
:1016800005020D430BE00F488078124940180F49BE
:10169000086008000068057801E00020E9E7C0461E
:1016A00004E0C0460020E4E70020E2E7C046074827
:1016B0008088A84201D905498D80FFF7E9FA012009
:1016C000D7E7000068010040941B00006001004063
:1016D000A61B0000EA1B000070B52E480078C0066B
:1016E000C00E04D0012808D002284ED11DE02A489F
:1016F0002A490860FFF7CCFA49E029480078002819
:101700000ED02448007927490978884208DA002158
:1017100025480170417021490860FFF7B9FA03E0DC
:10172000002070BC08BC184731E01A4804798F21AA
:101730000C408020044205D02107090F012000043D
:10174000884001E00120A0400500154800780028ED
:1017500002D12007000F15D114480068284211D08B
:1017600013480068284201D0012000E00020010455
:10177000090C0D480170090A417008490860FFF71B
:1017800087FA01E00020CCE701E00020C9E7C0466D
:101790000120C6E7680100404C01004060010040A4
:1017A0004F010040580100408801004050010040B6
:1017B0005401004070B5040033480078C006C00EE4
:1017C00004D0012821D0022859D120E02E48408899
:1017D000012815D1002C09D00120FFF745F82B482E
:1017E000008802210843294908800DE00020FFF706
:1017F0003BF826480088022188432449088003E0FA
:10180000002070BC08BC18473BE00020F9E71E48E8
:1018100005798F210D408020054205D02907090F49
:1018200001200004884001E00120A840060018487B
:101830000078002820D02807000F1DD01548006828
:10184000304219D010484088002813D1002C08D00D
:101850002800FFF77DF81048006830430E49086003
:101860000CE02800FFF783F80B480068B0430A49F2
:10187000086003E00020C4E70020C2E701E0002088
:10188000BFE7C0460120BCE7680100404C010040B2
:101890004F0100405001004054010040F8B55E483F
:1018A000807800287ED05D4C80E06078022804D0EB
:1018B000042852D0052873D151E0607956498978BF
:1018C000884243D154488078554908702079554959
:1018D0000870002603E0002053498855761C042E2A
:1018E000F9D3012615E00120B040504909680842AB
:1018F00002D03000FFF70EF801200004B0404B4941
:101900000968084204D0802131430800FFF702F83B
:10191000761C102EE7D3464844490860002045490C
:1019200008600120FEF7A1FFE079C021084206D03F
:1019300041480088012108433F4908800CE03E48A7
:101940000088400840003C49088005E0E078A17824
:1019500000020843041929E022E0E57820E0002D88
:101960001DD1A0788F21084006008020064205D0B6
:101970003107090F01200004884001E00120B04038
:1019800007002A4800683843284908602000FEF70D
:101990008CFF3000FEF7AFFF3000FEF7CAFFC046F5
:1019A000C04600E007E020780419C04620780028EF
:1019B00000D07AE724E0002019490870012615E0DC
:1019C0000120B04019490968084202D03000FEF7F2
:1019D000A1FF01200004B04014490968084204D066
:1019E000802131430800FEF795FF761C102EE7D3C7
:1019F0000F480E49086000200E490860FEF735FFC9
:101A00000548807806490978884203D10120F8BC4E
:101A100008BC18470020FAE768010040A61B000038
:101A20004F01004058010040590100405001004062
:101A300001000100540100404C010040F0B585B0A8
:101A400041480078002804D1002005B0F0BC08BC53
:101A50001847002000903D4C71E06078022804D0C7
:101A600004280ED0052866D11FE060793649097830
:101A7000884205D0E078A1780002084304195EE0AE
:101A800059E0A578E6780020029031480079A84214
:101A90000AD12F488078B04206D1012000902D480D
:101AA000405D03902B494E5545E029480079A842F6
:101AB00040D1A0788F2108400190802101980842F0
:101AC00006D001980107090F01200004884002E0B8
:101AD00001200199884007001D488078B04216D146
:101AE0001D48006838431C4908601C480068B8431A
:101AF0001A4908602000FEF7D8FE0198FEF7FBFEA9
:101B00000198FEF716FF02983843029012E00398FE
:101B100086420FD1029838420CD10F480068B84372
:101B20000D4908600D480068B8430C4908600198E9
:101B3000FEF7F0FEC046C04620780419C046207863
:101B400000288AD1009880E74F010040A61B0000C2
:101B5000680100405901004050010040540100401C
:101B6000000052E304309014042042120430811427
:101B7000FAFFFF1A1EFF2FE11EFF2FE10000A0E376
:101B8000000052E30420421204008114FBFFFF1AFC
:101B90001EFF2FE1120110010200004051C2051783
:101BA00000010420440109024300020100803209BF
:101BB000040000010202005E05240010010524015A
:101BC0000101042402020524060001070581031017
:101BD000000209040100020A00005E07050202403B
:101BE00000000705820240000000040309041C03F2
:101BF000450054005400200043004F002E002C00EC
:101C00004C00540044002E002000320345005400D4
:101C10002D00410052004D00370028004C005000BC
:101C20004300320033003600380029002000430012
:101C30006F006D0070006F00720074001A034400A2
:101C400045004D004F0030003000300030003000C3
:101C50003000300030000A03560043004F004D00B2
:101C60000D0D0000BF100000E71000000000000094
:101C70000000000000000000000000000000000064
:101C80000000000000000000000000000000000054
:101C90000000000000000000000000000000000044
:101CA000C01C000000000040880100000415000076
:101CB0001C1D000088010040D00600007C1B0000B5
:101CC0007201238025C20812C06AE0041A04041AB3
:101CD0000C045A14041A28045A0804291C200B184E
:101CE000F1FFFF18F2FFFF3C050253400A1602A461
:101CF0006C8007E0041A04041A0C045A14041A280D
:101D0000045A0804291C1A70A41A70A41AF0A431E9
:0C1D1000027C1029C849CA9201000000A2
:00000001FF
